:020000040000FA
:06000000703002303A28C6
:08000800A000030EA100831209
:1000100005191028831601178312B23081002B288E
:1000200083160113831203140B190310A80DA90DD5
:10003000AA0DAB0DAC0DAC16FF302C02031D2B2806
:10004000FA302B02031D2B2831152A08AF0029088E
:10005000AE002808AD008B100B11210E8300A00EFE
:04006000200E090065
:0C007400203084008001840A6030040207
:10008000031C3C281230B00058218316FF23900037
:10009000831283160C308505870183128501870141
:1000A000073099000030831691009F008312C830FA
:1000B00083168100831231309000003083168C004B
:1000C000831210308B00831600309B001C141A081A
:1000D0008312BC00831610309B001C141A08831274
:1000E000BD00952181018E018F010B118B100B102A
:1000F0008C018B178A2031198D203C21B30B882865
:10010000031085190314B90DF03039020319E520E5
:1001100098217A2864003210080031110130B700AC
:100120008B132030370783169B001C141A08831288
:10013000A4001030370783169B001C141A08831282
:10014000A300A6000230A6060030370783169B00E6
:100150001C141A088312A200A7000130A7068B17EF
:10016000321CB82822090339A200A309A409A50951
:1001700024082F02031DDF2823082E02031DCD288B
:1001800022082D02031DDF2801303702031DCD2870
:100190003D18CD283D143E146E2126082E02031D65
:1001A000DF2827082D02031DDF2801303702031D39
:1001B000DE283D1CDE283D103E149221DF28B70AC0
:1001C000023037020318080090280130B600B3004F
:1001D000B400B500B70085018701B1138A20B30BC5
:1001E0000B29031085190314B90DF03039020319D6
:1001F0003229B41F8501B41F8701B40B0B293708BE
:10020000B6080319B60003190929FF3085008700D5
:10021000B6039630B400311DEE283111321C152979
:100220002D090339AD00AE09AF092F1CEE288E0150
:100230008F010C1CEE280C102E1EEE288B13203084
:100240003707BB002F08BA00452110303707BB0025
:100250002E08BA00452100303707BB002D08BA0030
:1002600045218B1785018701B70AB6010230370295
:10027000031CEE28952108003E1C08003E1010309B
:10028000BB003D08BA00452108008B133A088316CD
:100290001C159A003B089B0055309D00AA309D001C
:1002A0009C1464009C1851291C1183128B170800A0
:1002B000831620309B001C141A088312DF00FF30C5
:1002C000D5000230D6000C30D700BA30D800373015
:1002D000D900DA30DA006F30DB0008000130BD00F1
:1002E0000430C200C5000530C400C600CA00073093
:1002F000C100C300C700C800C9005F19C1175F195A
:10030000C2175F19C317DF19C4175F1AC5175F1A21
:10031000C6175F1AC7175F1AC8175F1BC917DF1800
:10032000CA1708008501870108003D186E210800E2
:1003300001303D05031908005F19A0295C18051656
:100340005F19A429DC1885165F19A8295C19051402
:10035000DF19AC29DC1985145F1AB0295C1A8714DF
:100360005F1AB429DC1A07155F1AB8295C1B071439
:100370005F1ABC29DC1B87165F1BC0295D18071696
:10038000DF18C429DD188715E6300E02031CDC29AE
:100390005F1D05165F1D85165F1D0514DF1D851485
:1003A0005F1E87145F1E07155F1E07145F1E8716EA
:1003B0005F1F0716DF1C87158F08031908008F01C0
:1003C000850187015508DE00DA23D5005608DE00D6
:1003D000DA23D6005708DE00551CDA23D700580868
:1003E000DE00D51CDA23D8005908DE00551DDA23BB
:1003F000D9005A08DE00D51DDA23DA005B08DE00DA
:10040000551EDA23DB005F1D1F2AC11B1A2AC11CDF
:100410000512C11C0E2A051258190516CB0B302ADD
:100420005608CB00C101D51BC114D81BC1105818E8
:10043000C110302A0512CB0B302AC103302AC10863
:10044000031905160319302ACB0B302AD51BC1031B
:100450005508CB00D5185C14D51E5C10D51D5C105A
:100460005F1D4C2AC21B472AC21C8512C21C3B2A94
:10047000851258188516CC0B5D2A5608CC00C2018F
:10048000D61BC2145A18C210D619C2105D2A851282
:10049000CC0B5D2AC2035D2AC20803198516031915
:1004A0005D2ACC0B5D2AD61BC2035608CC00D61A97
:1004B000DC14561DDC10561FDC105F1D792AC31B8F
:1004C000742AC31C0510C31C682A05105A19051488
:1004D000CD0B8A2A5708CD00C301D71BC314D51AE8
:1004E000C310D719C3108A2A0510CD0B8A2AC3035B
:1004F0008A2AC3080319051403198A2ACD0B8A2AEC
:10050000D71BC3035708CD00571A5C15571F5C1142
:10051000D71D5C11DF1DA62AC41BA12AC41C85108F
:10052000C41C952A8510D51B8514CE0BC22A5808E9
:10053000CE00C401D81BC414D71AC410D819C410D3
:10054000C22A8510CE0BC22AC403C22ADF1FB12AD9
:10055000CE0BC22A5808CE00D51BDC15DA1FDC11E1
:10056000C22AC408031985140319C22ACE0BC22A51
:10057000D81BC4035808CE00581ADC15D81FDC114C
:10058000D81DDC115F1EDE2AC51BD92AC51C8710A9
:10059000C51CCD2A8710D51A8714CF0BEF2A59080E
:1005A000CF00C501D91BC514561AC510D81BC510DC
:1005B000EF2A8710CF0BEF2AC503EF2AC5080319CE
:1005C00087140319EF2ACF0BEF2AD91BC50359084B
:1005D000CF00D91B5C16D91F5C12D91C5C125F1EA0
:1005E0000B2BC61B062BC61C0711C61CFA2A0711AB
:1005F000D71A0715D00B1C2B5A08D000C601DA1BDE
:10060000C614D51AC610D619C6101C2B0711D00B4C
:100610001C2BC6031C2BC6080319071503191C2B1A
:10062000D00B1C2BDA1BC6035A08D0005A1ADC1652
:100630005A1EDC12DA1FDC125F1E382BC71B332B4D
:10064000C71C0710C71C272B071059190714D10BFB
:10065000492B5B08D100C701DB1BC714D719C71092
:10066000DB19C710492B0710D10B492BC703492BA6
:10067000C708031907140319492BD10B492BDB1B9E
:10068000C7035B08D100DB195C17DB1D5C135B1E25
:100690005C135F1E652BC81B602BC81C8712C81C0F
:1006A000542B871258198716D20B762B5608D20076
:1006B000C801D91BC8145A19C810551AC810762B6E
:1006C0008712D20B762BC803762BC808031987161E
:1006D0000319762BD20B762BD71BC8035908D200EF
:1006E000561ADC17561EDC13DA1FDC135F1F922B21
:1006F000C91B8D2BC91C0712C91C812B0712551948
:100700000716D30BAC2B5808D300C901D61BC9144C
:10071000D91AC910D819C910AC2B0712D30BAC2B9E
:10072000C903AC2B5F1C9D2BD30BAC2B5708D300FC
:10073000D61B5D14D81F5D10AC2BC9080319071612
:100740000319AC2BD30BAC2BD51AC9035808D30013
:10075000D61B5D14D81F5D10DF1CC82BCA1BC32B12
:10076000CA1C8711CA1CB72B8711D51B8715D40B40
:1007700008005508D400CA01D51BCA14561ACA105D
:10078000D619CA1008008711D40B0800CA03080044
:10079000CA080319871503190800D40B0800D81BD1
:1007A000CA035608D400591ADD14591EDD10DA1F89
:1007B000DD100800C001DE080319DE035E184014D6
:1007C000DE1A40144008C0015E1C4014DE1E4014B6
:0807D000C005C00C5E0C08001E
:084000000D000300040008009C
:02400E00CC01E3
:10420000010078007A007C007E007B0079007F004E
:104210007D007A0078007E007C00FF00FF00FF0038
:104220000100F200F600FA00FE00F200F600FA00CB
:10423000FE00F200F600FA00FE00FF00FF00FF00A3
:10424000030005000500050005000900090009003C
:1042500009000D000D000D000D00FF00FF00FF0024
:10426000FF00FF00FF00FF00FF00FF00FF00FF0056
:10427000FF00FF00FF00FF00FF00FF00FF00FF0046
:10428000FF00FF00FF00FF00FF00FF00FF00FF0036
:10429000FF00FF00FF00FF00FF00FF00FF00FF0026
:1042A000FF00FF00FF00FF00FF00FF00FF00FF0016
:1042B000FF00FF00FF00FF00FF00FF00FF00FF0006
:1042C000FF00FF00FF00FF00FF00FF00FF00FF00F6
:1042D000FF00FF00FF00FF00FF00FF00FF00FF00E6
:1042E000FF00FF00FF00FF00FF00FF00FF00FF00D6
:1042F000FF00FF00FF00FF00FF00FF00FF00DD00E8
:00000001FF
